:04000000B2017129AF
:10000800B216B21EB212B2190D28B2154620031844
:1000180034280830A3005A20A20DA30B0F28B21EC3
:100028003F2064206020B21A3420392022080310AF
:100038006C29B216B21EB21232192728FE39B30043
:10004800321503106C29321A2F28A60032164620C2
:100058000318342826084D2003183428B21E6C29AA
:100068003F20642032113212B2113608840034085D
:1000780084178004452836088400340980058417CD
:1000880080050800392064203F2060203308B21919
:100098000138A2000830A300A20D03183920031C60
:1000A8003F2064206020A30B5028392064203608A4
:1000B800840034080005FF3E3708840035094228CB
:1000C8003708840035083C280408A6003608840050
:1000D8008030B3050830A70003100318B30A822044
:1000E800A60CA70B71280000AB1A330C82206F21D5
:1000F800031482202F08A3002E0824298413AB1F81
:100108009128000834042B1F340680008417000847
:100118003404031C340680009C2800083404031CA3
:1001280034062B1B340680008417340980059C286C
:100138002B081F39003EA1002A08083E0318A10A0F
:1001480000003129B31329080319B3170430A80094
:10015800250EB3202508B320240EB32024080F3918
:10016800F63E0318073E0A3EB928A000A803031963
:10017800B31329080319C328280203180800200804
:10018800031DB313B31B0800303E67290830A600CF
:10019800A70037088400350833191721331D1921A2
:1001A8003608840034081C21A001A101260803197F
:1001B8006C29B3180E213608840000083405FF3E68
:1001C800A00DA10DB31C0E21A60BDD28270833189E
:1001D800452920086C290830A6003708840035080E
:1001E80033191721331D19213608840034092021B9
:1001F800260803196C293318452136088400A10CF8
:10020800A00C00083404031C340680000E21A60B41
:1002180001296C2937088400350880060000142954
:1002280015298006080080041F29FF3A8005202927
:10023800841780046C29FF3A841780056C29A30170
:10024800A200FF30A207031CA307031C6C2903307C
:10025800A100E43031212529A101F63EA000A10921
:10026800031C3C29FE300000A00703183729A0070B
:100278006400A10F362900002018422920184429BB
:100288000800A201A3014C29A10CA00CA20DA30DEA
:10029800FF3E031848292308A1002208A0006C2962
:1002A800A20001305729A80023082102031D5E2956
:1002B80022082002043003180130031902302805EF
:1002C800031DFF306C29840031088A003008820041
:1002D80083130313831264000800831607309F00FA
:1002E8008312FA010430FB00FC01EA30FD0083169A
:1002F800D1010830C4008312E2011030E300043059
:10030800F200F301F4011030F5008316B401B501D1
:1003180090308700B001B1018312DE01DF01E001F6
:10032800E101D801D9010130A300F4308A01242168
:100338000730B6004030B4002030AA00AB01AE014F
:10034800AF0153308A01692074308A016920613015
:100358008A01692072308A01692074308A01692013
:100368000A308A0169200D308A0169208A110A122F
:10037800D52E07148316FF30C7000130CF00831233
:1003880064000B3083164F028A110A128312031875
:10039800E5290730B6002030B4000730B700083030
:1003A800B5000130B300831647088312A000A101ED
:1003B8008A01EF208316CF0A8A110A128312031DBD
:1003C800C429071032308A01232183164030C50022
:1003D800BC01BD01BE01BF019530C6008312831662
:1003E8004508C70007308312B6002030B400073034
:1003F800B7000830B5000130B300831647088312F0
:10040800A000A1018A01EF2083163C08C70007302D
:100418008312B6002030B4000730B7000830B500AA
:100428000130B300831647088312A000A1018A0196
:10043800EF2083163D08C70007308312B60020302E
:10044800B4000730B7000830B5000130B300831698
:1004580047088312A000A1018A01EF2083163E08F5
:10046800C70007308312B6002030B4000730B70049
:100478000830B5000130B300831647088312A00086
:10048800A1018A01EF2083163F08C70007308312B5
:10049800B6002030B4000730B7000830B50001308E
:1004A800B300831647088312A000A1018A01EF2038
:1004B80083164608C70007308312B6002030B40000
:1004C8000730B7000830B5000130B300831647087D
:1004D8008312A000A1018A01EF206400831652084C
:1004E800013C8A110A12831203198A2A0730B600BE
:1004F8001030B4000730B7000830B500B3018A01E6
:10050800CA208316D20083128A01712A0714323056
:100518008A0123210710640083165208003C8A11BF
:100528000A12831203194F2B07148316FF30C700D2
:1005380007308312B6002030B4000730B700083007
:10054800B5000130B300831647088312A000A1014B
:100558008A01EF200730B6001030B4000730B7002A
:100568000830B500B3018A01CA208316D20083126D
:10057800071083164130C70007308312B6002030B9
:10058800B4000730B7000830B5000130B300831657
:1005980047088312A000A1018A01EF208316C70132
:1005A80007308312B6002030B4000730B700083097
:1005B800B5000130B300831647088312A000A101DB
:1005C8008A01EF200730B6002030B4000730B700AA
:1005D8000830B5000130B300831647088312A00025
:1005E800A1018A01EF200730B6002030B40007309F
:1005F800B7000830B5000130B300831647088312EE
:10060800A000A1018A01EF200730B6002030B40015
:100618000730B7000830B5000130B300831647082B
:100628008312A000A1018A01EF208316FF30C700C2
:1006380007308312B6002030B4000730B700083006
:10064800B5000130B300831647088312A000A1014A
:100658008A01EF200730B6002030B4000730B70019
:100668000830B5000130B300831647088312A00094
:10067800A1018A01EF200730B6001030B40007301E
:10068800B7000830B500B3018A01CA208316D2002A
:1006980083128A018F2A0730B6004030B400203018
:1006A800AA00AB01AE01AF0149308A0169204E3082
:1006B8008A01692049308A01692054308A016920F9
:1006C80020308A0169204F308A0169204B308A0125
:1006D80069200A308A0169200D308A016920831651
:1006E800FF30C7008312080007148316FF30C700C5
:1006F80007308312B6002030B4000730B700083046
:10070800B5000130B300831647088312A000A10189
:100718008A01EF200730B6001030B4000730B70068
:100728000830B500B3018A01CA208316D2008312AB
:10073800071083165830C70007308312B6002030E0
:10074800B4000730B7000830B5000130B300831695
:1007580047088312A000A1018A01EF200730B600E4
:100768002030B4000730B7000830B5000130B300BE
:100778005B08A000A1018A01EF200730B6002030F5
:10078800B4000730B7000830B5000130B3005A088C
:10079800A000A1018A01EF200730B6002030B40084
:1007A8000730B7000830B5000130B3005D08A0007D
:1007B800A1018A01EF200730B6002030B4000730CD
:1007C800B7000830B5000130B3005C08A000A101F3
:1007D8008A01EF208316FF30C70007308312B60066
:1007E8002030B4000730B7000830B5000130B3003E
:1007F800831647088312A000A1018A01EF20073061
:10080800B6001030B4000730B7000830B500B301A7
:100818008A01CA208316D200831264008316520804
:10082800003C8A110A12831203192A2C0730B600D9
:100838001030B4000730B7000830B500B3018A01A2
:10084800CA208316D20083128A01112C8316FE3027
:10085800C70007308312B6002030B4000730B70055
:100868000830B5000130B300831647088312A00092
:10087800A1018A01EF206408D8006508D90058084A
:10088800A0005908A1006708A30066088A0154213E
:100898008A110A12031D962C0730B6000230B400E4
:1008A8000730B7000430B500A0308A011F2059086E
:1008B8008A011F2058088A011F208A0104208316F4
:1008C800C70007308312B6002030B4000730B700E5
:1008D8000830B5000130B300831647088312A00022
:1008E800A1018A01EF200730B6004030B400203063
:1008F800AA00AB01AE01AF010230A9008316470878
:100908008312A400A5016830B000B1018A01A620B5
:1009180020308A016920D80A0319D90A8A110A12D3
:10092800031D432C8316FF30C70007308312B6001F
:100938002030B4000730B7000830B5000130B300EC
:10094800831647088312A000A1018A01EF2007300F
:10095800B6002030B4000730B7000830B5000130C9
:10096800B300831647088312A000A1018A01EF2073
:100978000730B6001030B4000730B7000830B500B3
:10098800B3018A01CA208316D2000F305205D50060
:1009980007308312B6001030B4000730B7000830B3
:1009A800B500B3018A01CA208316D20083126400FD
:1009B80083165208003C8A110A128312031DF42C74
:1009C8000730B6001030B4000730B7000830B50063
:1009D800B3018A01CA208316D20083128A01DB2C54
:1009E8008A110A12E425080007148316FF30C7008D
:1009F80007308312B6002030B4000730B700083043
:100A0800B5000130B300831647088312A000A10186
:100A18008A01EF200730B6001030B4000730B70065
:100A28000830B500B3018A01CA208316D2008312A8
:100A3800071083165130C70007308312B6002030E4
:100A4800B4000730B7000830B5000130B300831692
:100A580047088312A000A1018A01EF200730B600E1
:100A68002030B4000730B7000830B5000130B300BB
:100A78005B08A000A1018A01EF200730B6002030F2
:100A8800B4000730B7000830B5000130B3005A0889
:100A9800A000A1018A01EF200730B6002030B40081
:100AA8000730B7000830B5000130B3005D08A0007A
:100AB800A1018A01EF200730B6002030B4000730CA
:100AC800B7000830B5000130B3005C08A000A101F0
:100AD8008A01EF208316FF30C70007308312B60063
:100AE8002030B4000730B7000830B5000130B3003B
:100AF800831647088312A000A1018A01EF2007305E
:100B0800B6001030B4000730B7000830B500B301A4
:100B18008A01CA208316D200831264008316520801
:100B2800003C8A110A1283120319AA2D0730B60055
:100B38001030B4000730B7000830B500B3018A019F
:100B4800CA208316D20083128A01912D640083166D
:100B58005208FE3C8A110A1283120319C32D07306A
:100B6800B6001030B4000730B7000830B500B30144
:100B78008A01CA208316D20083128A01AA2D08008E
:100B88000730B6001030B4000730B7000830B500A1
:100B9800B3018A01CA208316D20007308312B60037
:100BA8001030B4000730B7000830B500B3018A012F
:100BB800CA208316D20083128A110A12E42508007B
:100BC80007148316FF30C70007308312B6002030A1
:100BD800B4000730B7000830B5000130B300831601
:100BE80047088312A000A1018A01EF200730B60050
:100BF8001030B4000730B7000830B500B3018A01DF
:100C0800CA208316D2008312071083164D30C700FE
:100C180007308312B6002030B4000730B700083020
:100C2800B5000130B300831647088312A000A10164
:100C38008A01EF208316C70107308312B6002030DF
:100C4800B4000730B7000830B5000130B300831690
:100C580047088312A000A1018A01EF200730B600DF
:100C68002030B4000730B7000830B5000130B300B9
:100C7800831647088312A000A1018A01EF200730DC
:100C8800B6002030B4000730B7000830B500013096
:100C9800B300831647088312A000A1018A01EF2040
:100CA8000730B6002030B4000730B7000830B50070
:100CB8000130B300831647088312A000A1018A01FE
:100CC800EF208316FF30C70007308312B6002030AC
:100CD800B4000730B7000830B5000130B300831600
:100CE80047088312A000A1018A01EF200730B6004F
:100CF8001030B4000730B7000830B500B301103029
:100D08008A01CB208316AE00831221088316AF0018
:100D18002E08D10083120800831640088312DB00D6
:100D2800831641088312DA00831642088312DD0015
:100D3800831643088312DC000800E401E501FF3054
:100D4800E6000130E700DA01DB01DC01DD018A01A0
:100D580078230800E4010230E500FF30E6000330A4
:100D6800E7000330DA00DB01DC01D030DD008A0166
:100D780078230800E4011030E500FF30E600113068
:100D8800E700DA01DB01DC010430DD008A017823A9
:100D98000130DA00DB01DC01EA30DD008A0178236A
:100DA8000800E401E501FF30E6000130E700DA0160
:100DB800DB01DC01DD018A01BD21D801D901580818
:100DC800A0005908A100A3017F308A0154218A118B
:100DD8000A12031DA42F59088A110A12031D872F0E
:100DE80058087F3C8A110A12031C872F8A110A129D
:100DF80003278316C70083128A110A12872F073028
:100E08008A0058088207EB343C3490344D3453340C
:100E180044344F34533435342E34303400340234AF
:100E2800083402340034023400340234003400340C
:100E3800F834F33400343F340034FF34003465347C
:100E48000034003400349B349934073400340034BF
:100E5800003429343C345634C63460344E344F346C
:100E680020344E3441344D34453420342034203439
:100E78002034463441345434313436342034203428
:100E880020343334C9348E34D134BC34F0347B3418
:100E98008E34D934B834003420348E34C034FC3421
:100EA800BD3400347C3438344E3424347D34243416
:100EB8008B34C1349934E8343C34013472341C34F2
:100EC8008334EB343A346634A1341C347C3426340D
:100ED80066343B34073426348A345734FC3475344A
:100EE80006348034CA3402348834563402348034A8
:100EF800C33410347334EB343334C9348A3446344D
:100F080010349834F7340730B6000230B400073094
:100F1800B7000430B500A0308A011F2059088A01A3
:100F28001F2058088A011F208316470883128A0148
:100F38001D20D80A0319D90A8A110A12031DE32EA3
:100F48008030D800D9018316BA01BB0183128316F9
:100F58003A088312A00083163B088312A100A3015C
:100F68007F308A0154218A150A12031DA32883168B
:100F78003B088A150A128312031D812883163A0832
:100F88007F3C8A150A128312031C81288A110A12CF
:100F9800D3278316C70083128A150A1281280830BE
:0A0FA8008A0083163A08831200281D
:10100000820766341634033446341C3413345634A1
:101010001E34033446340E341334D1348B347634D6
:101020001134603489344634FC3489345634FE3407
:10103000B83420340034F734E6348B345E340B3467
:101040000334C3344834F734F33401344634FC34C5
:1010500011344E34FE346134BF3400340034E8348B
:10106000E634003472343934263438342D34743450
:1010700017346034B1340B34BE34A1347D34F334CE
:10108000A6346134743432344E34743409348334C5
:10109000C73420343B34FB347234E634EB34DC3474
:1010A000A034FB347D34B4347D348B34F034AC3430
:1010B0009834403474340C34483474341334B434B5
:1010C0000E34BB3407340034CD341034EB34EF34F9
:1010D000A034FD347D34EB34E634A034FC347D346C
:1010E000EB34E134CD341634CD34193426348B341A
:1010F00055341A345234B0340134BB340034003423
:10110000E8340730B6000230B4000730B7000430CE
:10111000B500A0308A011F2059088A011F205808F5
:101120008A011F208316470883128A011D20D80ACE
:101130000319D90A8316BA0A0319BB0A8A110A12BB
:101140008312031DAB2FD8010130D9008316BA01D9
:10115000BB01831283163A088312A00083163B0852
:101160008312A100A3017F308A0154218A150A123B
:10117000031DA32983163B088A150A128312031D37
:10118000812983163A087F3C8A150A128312031CB0
:1011900081298A150A12D2208316C70083128A1564
:1011A0000A12812909308A0083163A08831200291D
:1012000082073B3400347234E8345B348A34563419
:101210002434BE340B347C348B34FC34C734463431
:10122000F0343D347D34C7344634F43429347D34CD
:101230008C34D93489344E34F23489344E34F63413
:10124000C634063496347D34CB34EA340334003467
:10125000003420340F34B634C83466348B3446340A
:10126000F8346634033446341C3466348B34D0345A
:101270006634C134EA341034EB345E340F34B6349F
:10128000C8344A344A348A3446340D343234E4346F
:10129000F734E23403344634FC3413345634FE3429
:1012A000EB344A3452345034063453346A34013403
:1012B0006A34103491348B34463418349634923472
:1012C0003334D234F734F6349134F734F6344234CC
:1012D0008734CA34F73476341A348A34F2348A3490
:1012E000E834C034CC3402340A34CC34B834013459
:1012F000023480347E3402340E3475340434B43411
:1013000042340730B6000230B4000730B700043072
:10131000B500A0308A011F2059088A011F205808F3
:101320008A011F208316470883128A011D20D80ACC
:101330000319D90A8316BA0A0319BB0A8A150A12B5
:101340008312031DAA288030D8000130D9008316EB
:10135000BA01BB01831283163A088312A0008316D8
:101360003B088312A100A3017F308A0154218A1512
:101370000A12031DA32A83163B088A150A12831238
:10138000031D812A83163A087F3C8A150A128312AC
:10139000031C812A8A150A12D3218316C7008312DF
:1013A0008A150A12812A0A308A0083163A088312A3
:0213B000002A11
:1014000082078B34F4348A3456342434CD34133484
:101410006134613472340B344034753401344234F5
:1014200003345E340B34493475340634F834C33431
:101430004134BB3400340034603466346A340034E0
:10144000EB34B0344E3454344C34443452342034BD
:10145000203420342034203420340D340A345234E3
:1014600065346D346F3476346534203464346934D3
:1014700073346B34733420346F34723420346F34EB
:10148000743468346534723420346D3465346434B3
:10149000693461342E34FF340D340A3444346934F1
:1014A00073346B3420346534723472346F34723474
:1014B000FF340D340A345034723465347334733469
:1014C000203461346E34793420346B3465347934AB
:1014D000203474346F34203472346534733474348B
:1014E0006134723474340D340A34003400340034FE
:1014F0000034003400340034AC34CB34D8345534A8
:10150000AA340730B6000230B4000730B700043008
:10151000B500A0308A011F2059088A011F205808F1
:101520008A011F208316470883128A011D20D80ACA
:101530000319D90A8316BA0A0319BB0A8A150A12B3
:101540008312031DAB290730B6004030B4002030B1
:10155000AA00AB01AE01AF0142308A0169206F30B1
:101560008A0169206F308A01692074308A016920FC
:1015700020308A01692074308A0169206F308A0125
:10158000692020308A01692065308A016920653030
:101590008A01692070308A01692072308A016920CD
:1015A0006F308A0169206D308A0169200A308A0112
:1015B00069200D308A0169200730B6000230B4007E
:1015C0000730B7000430B500A0308A011F2010306A
:1015D0008A011F2000308A011F20F8308A011D2057
:1015E0000730B6000230B4000730B7000430B50051
:1015F000A0308A011F2010308A011F2001308A018B
:101600001F20FF308A011D200730B6000230B400D1
:101610000730B7000430B500A0308A011F20103019
:101620008A011F2002308A011F20FF308A011D20FD
:101630000730B6000230B4000730B7000430B50000
:10164000A0308A011F2010308A011F2003308A0138
:101650001F20FF308A011D200730B6000230B40081
:101660000730B7000430B500A0308A011F201030C9
:101670008A011F2004308A011F20FF308A011D20AB
:101680000730B6000230B4000730B7000430B500B0
:10169000A0308A011F2010308A011F2005308A01E6
:1016A0001F20FF308A011D200630D8001030D900DD
:1016B0005808A0005908A1001130A300FF308A018A
:1016C00054218A150A12031D802B0730B600023000
:1016D000B4000730B7000430B500A0308A011F20E5
:1016E00059088A011F2058088A011F2000308A01EA
:1016F0001D20D80A0319D90A8A150A12031D582B6E
:10170000D8010230D9008316BA01BB0183128316B7
:101710003A088312A00083163B088312A100A3019C
:101720003F308A0154218A150A12031D172C831693
:101730003B088A150A128312031DF52B83163A08FB
:101740003F3C8A150A128312031CF52B8A150A12D4
:10175000AF238316C70083128A150A12F52B0B30AC
:101760008A0083163A0883128207E53445345334DD
:10177000543444344134543441345434583454345B
:10178000203418344234033498348F3433348F3453
:10179000333400340034043498348F343334003418
:1017A00000340034003400340034543445345334AD
:1017B000543444344134543441345434583454341B
:1017C000203418344234033498348F3433348F3413
:1017D0003334003400345D3498348F34333402347D
:1017E000003400340034003400340730B6000230D6
:1017F000B4000730B7000430B500A0308A011F20C4
:1018000059088A011F2058088A011F20831647089B
:1018100083128A011D20D80A0319D90A8316BA0A2D
:101820000319BB0A8A150A128312031D872B403045
:10183000D8000230D9005808A0005908A100033090
:10184000A300FF308A0154218A150A12031D432C7C
:101850000730B6000230B4000730B7000430B500DE
:10186000A0308A011F2059088A011F2058088A01C8
:101870001F2000308A011D20D80A0319D90A8A15B1
:101880000A12031D1B2C0730B6004030B400203074
:10189000AA00AB01AE01AF0145308A016920653075
:1018A0008A01692070308A01692072308A016920BA
:1018B0006F308A0169206D308A01692020308A01E9
:1018C00069206C308A0169206F308A01692061309B
:1018D0008A01692064308A01692065308A016920A3
:1018E00064308A0169200A308A0169200D308A013A
:1018F00069208A01A1260730B6004030B4002030AC
:10190000AA00AB01AE01AF0142308A0169206F30FD
:101910008A0169206F308A01692074308A01692048
:1019200020308A01692073308A01692061308A0180
:10193000692076308A01692065308A016920643027
:101940008A0169200A308A0169200D308A016920E4
:101950008A01BE260730B6004030B4002030AA000D
:10196000AB01AE01AF0146308A01692041308A01E6
:10197000692054308A01692020308A01692073303F
:101980008A01692061308A01692076308A016920E4
:1019900065308A01692064308A0169200A308A0131
:1019A00069200D308A0169208A01AE268316BA01AA
:1019B000BB01831283163A088312A00083163B08EA
:1019C0008312A1000130A300FF308A0154218A153F
:1019D0000A12031D262D0730B6000230B40007306E
:1019E000B7000430B500A0308A011F2083163B08E1
:1019F00083128A011F2083163A0883128A011F204E
:101A00008A0104208316C70007308312B6004030D5
:101A1000B4002030AA00AB01AE01AF010230A90032
:101A2000831647088312A400A5016830B000B101F5
:101A30008A01A62020308A0169208316BA0A031978
:101A4000BB0A8A150A128312031DDA2C0730B6006E
:101A50004030B4002030AA00AB01AE01AF014430E9
:101A60008A01692049308A01692052308A0169203F
:101A700020308A01692053308A01692061308A014F
:101A8000692076308A01692065308A0169206430D6
:101A90008A0169202E308A0169202E308A0169204E
:101AA0002E308A01692044308A0169204F308A0132
:101AB00069204E308A01692045308A016920213031
:101AC0008A0169200A308A0169200D308A01692063
:101AD00064008A150A12682D63008A150A126C2D9B
:02400E003D3D36
:00000001FF
